S123E000FEA0006E008D406E00101604BDE3348D67815326FA8D6181392729813126F07F90
S123E020A00F8D318002B7A0478D1C8D287AA0472709A700A10026080820F07CA00F27CFB1
S123E040863F8D317EE2D48D0CB7A00D8D07B7A00EFEA00D398D5348484848168D4C1B160B
S123E060FBA00FF7A00F3944444444840F8B30813923028B077EE1D17EE1AC8DF808A600D6
S123E080810426F7397EE14A8DBDCEE19D8DEFCEA00D8D34FEA00D8D318D318DDB81202753
S123E0A0FA810D27E0815E202C018DCC80302B4C81092F0A81112B4481162E40800739A6F2
S123E0C0008DA4A6000820A38DF58DF3862020A58EA040202C26070909FFA00D20ACFFA01D
S123E0E00D2002206D813025A18146229D8DBDBDE05709A700A10027917EE040BEA00820F8
S123E10049BFA00886FFBDE308CE8004BDE284A600A1022002201926398603A7008611A738
S123E12000202F01BFA008306D0626026A056A06CEE19DBDE07EFEA008088D8E8D8C8D8A1A
S123E1407EE35F01CEA008BDE0C8FEA0128CE12327198EA040CE8004FFA00A7FA00C8D730B
S123E1602703BDE27DBDE353BDE347CEE19CBDE07E8D39CEE3D1A1002607BDE0CCEE016E39
S123E180000808088CE3F826ED20BFFEA0126E005339040D0A15000000533104130D0A1569
S123E1A00000002404204CFEA0066E002040BDE047FFA004BDE047BDE05516A600FFA00D90
S123E1C01127022021CEE19DBDE07ECEA00D20103B203AFFA010FEA00A37E601E103333954
S123E1E0BDE0C8FEA00DBCA004279E0820CD8D06847F39313131378DDA26288615A700A6BB
S123E200004724FBA601F6A00C27072011378DC3262EC611E700E600575724FAA70133FEC8
S123E220A01039A6002BFC8D3AC604E702588D2A0D6900465A26F78D21F6A00C271320DEE0
S123E2408D23C60A6A008D168D10A7000D465A26F7E602582AC88D0220C46D022AFC6C0277
S123E2606A02396F028DF720F18D83167FA00BFEA00A8D108D07CEE3EF177EE1768634A7D9
S123E28003A702396C008607A7016C00A702397F80148D2EC60B8D25E604C50126FA6F0610
S123E2A08D1DC69C8D17CE2400C5022706B6801BA70008F68018C50126EF7E2400E7048D41
S123E2C00039CEFFFF098C801426FA39CEE009BDE07E8DF1BDE3472058CEE123BCA012279D
S123E2E01A088D32BDE047FFA014A600B7A016863FA700CEE1238D1E7EE16BFEA014B6A0D4
S123E30016A700CEE12420DAB7A041FEA0128CE1232706CEE124FFA012398D5A200FCEA029
S123E32049FFA004098D52CEE190BDE07E8D248D917EE15273A00C8611C6208D1ABDE1D971
S123E3402704863CA703398613C610200A8612C60420048614C608BDE075BDE1D62016BDE9
S123E360E0C8BDE0C8BDE0C87EE144E7008D028606A701E70039FEA002FFA0448DCFB6A085
S123E38005B0A045F6A004F2A044260481102502860F8B04B7A0478003B7A046CEE193BDAC
S123E3A0E07E5FCEA0478D24CEA0448D1F8D1DFEA0448D187AA04626F9FFA0445337308DFE
S123E3C00B33FEA04409BCA00426B339EB007EE0BF47E1D05AC0004DE08846E1AE52E13097
S11BE3E04AE00543E2CC44E28F42E2D94FE26950E31A4CE00C45E31EEA
S10BE3F8E000E18BE1A7E0D095
S105A048E0D062
S9030000FC
